:100000000C9434000C9446000C9446000C9446006A
:100010000C9446000C9446000C9446000C94460048
:100020000C9446000C9446000C9446000C94460038
:100030000C9446000C9446000C941B010C94460052
:100040000C9446000C9446000C9446000C94460018
:100050000C9446000C9446000C9446000C94460008
:100060000C9446000C94460011241FBECFEFD8E03C
:10007000DEBFCDBF11E0A0E0B1E001C01D92AE3106
:10008000B107E1F70E940B030C94D2030C9400001B
:10009000DF93CF93CDB7DEB7A4E2B0E0E4E2F0E0C7
:1000A000808180628C93A5E2B0E0E5E2F0E080819F
:1000B00080628C93A5E4B0E0E5E4F0E08081877F86
:1000C0008C93A4E4B0E0E4E4F0E0808182608C935F
:1000D000A4E4B0E0E4E4F0E080818E7F8C93E7E478
:1000E000F0E08CE98083AEE6B0E0EEE6F0E08081FF
:1000F00082608C93A5E4B0E0E5E4F0E08081846068
:100100008C93A5E4B0E0E5E4F0E080818D7F8C93F2
:10011000A5E4B0E0E5E4F0E0808181608C93AFE598
:10012000B0E0EFE5F0E0808180688C9388EC90E0AF
:100130009093140180931301809113019091140105
:100140000097D1F7A8E2B0E0E8E2F0E080818E7F8E
:100150008C9381E080931C01A7E2B0E0E7E2F0E03D
:1001600080818B7F8C931092000110920F0110926E
:1001700002011092010110921601109215011092C5
:1001800007011092060110921801109217011092A7
:10019000080110921D01109211011092100110928D
:1001A0000E0110920D01A5E2B0E0E5E2F0E08081E1
:1001B0008F7D8C931092040110920301E6E2F0E02F
:1001C0008081882F90E084709070009771F4109275
:1001D000120110920C0110920B010E94E2020E9487
:1001E000020381E080930F0123C081E0809312011C
:1001F0000E94BA0280910B0190910C01843091050C
:1002000038F080910B0190910C01893C910530F000
:100210008CE090E090930C0180930B0180910B0196
:1002200090910C0190930401809303010E94E202DB
:10023000CF91DF9108951F920F920FB60F92112464
:100240002F933F938F939F93AF93BF93EF93FF931E
:10025000DF93CF9300D000D00F92CDB7DEB780915F
:100260000F0180930001E6E2F0E08081882F90E0AA
:10027000847090701D82009711F421E02D833D81E0
:1002800030930F0180910001882339F480910F0190
:10029000813019F481E0809319018091120182303C
:1002A000B9F4E6E2F0E08081882F90E084709070ED
:1002B000009751F480910D0190910E010196909359
:1002C0000E0180930D0104C010920E0110920D01D9
:1002D00080911C01882F90E00097D1F48091090152
:1002E00090910A01009751F08091090190910A01C3
:1002F000019790930A01809309010AC0A8E2B0E037
:10030000E8E2F0E080818E7F8C9381E080931C0195
:1003100080910501282F30E03C832B838B819C81C9
:100320008130910519F12B813C812230310509F48E
:100330003EC08B819C81009709F06BC080910301C6
:1003400090910401009709F464C082E08093050154
:100350008EE190E09093180180931701A5E2B0E040
:10036000E5E2F0E080818F7D8C9353C0809106019F
:1003700090910701009751F080910601909107013B
:100380000197909307018093060143C082E0809318
:1003900005018EE190E09093180180931701A5E28A
:1003A000B0E0E5E2F0E080818F7D8C9332C08091F7
:1003B000170190911801009751F0809117019091C9
:1003C00018010197909318018093170122C0809122
:1003D0000301909104010097D1F081E08093050121
:1003E00084E090E09093070180930601A5E2B0E0DD
:1003F000E5E2F0E0808180628C938091030190912E
:1004000004010197909304018093030102C01092AC
:1004100005018091130190911401009749F080919A
:10042000130190911401019790931401809313018B
:100430008091100190911101009749F08091100175
:100440009091110101979093110180931001809177
:1004500001019091020101969093020180930101A4
:10046000809101019091020123E0883E920708F4F7
:100470003EC010920201109201018091120182305F
:10048000B1F5809115019091160101969093160196
:100490008093150180910801813039F480911A010F
:1004A00090911B019A83898306C020910B013091A2
:1004B0000C013A83298380911501909116012981BD
:1004C0003A818217930798F0109216011092150145
:1004D000A8E2B0E0E8E2F0E0808181608C938CE2F9
:1004E00091E090930A018093090110921C010F90F2
:1004F0000F900F900F900F90CF91DF91FF91EF91A0
:10050000BF91AF919F918F913F912F910F900FBE0F
:100510000F901F901895DF93CF93CDB7DEB7F89467
:10052000EFE3F0E08081882F90E082709070009778
:10053000B9F7E2E4F0E01082E1E4F0E01082E0E4F8
:10054000F0E080910B0190910C018083AFE3B0E06B
:10055000EFE3F0E080818F7D8C93AFE3B0E0EFE3D9
:10056000F0E080818F7E8C93FA9AF99A7894CF91FB
:10057000DF910895DF93CF93CDB7DEB7F894EFE323
:10058000F0E08081882F90E0827090700097B9F73A
:10059000E2E4F0E01082E1E4F0E01082AFE3B0E0EA
:1005A000EFE3F0E0808181608C93E0E4F0E0808113
:1005B000882F90E090930C0180930B017894CF9159
:1005C000DF910895DF93CF93CDB7DEB780910B0114
:1005D00090910C01969587959695879590931B0120
:1005E00080931A0180911A0190911B01843091052A
:1005F00030F484E090E090931B0180931A01CF9136
:10060000DF910895DF93CF93CDB7DEB71092190134
:10061000CF91DF910895DF93CF9300D000D00F9258
:10062000CDB7DEB70E94480080911201282F30E03C
:100630003D832C838C819D8181309105B9F02C8183
:100640003D812230310534F48C819D81009709F47D
:100650005CC0EACF2C813D8122303105B9F08C811C
:100660009D818330910509F440C0DECF8091050162
:100670008823D1F680910301909104010097A1F69F
:1006800082E0809312010E940203CECF8091190173
:100690008823F9F00E940203809108011B828130B7
:1006A00011F091E09B832B81209308018091080138
:1006B000813029F483E090E09A83898304C022E0AA
:1006C00030E03A83298389819A8190930401809351
:1006D000030180910D0190910E01883C910508F471
:1006E000A3CF83E0809312019FCF10921C0188EC6E
:1006F00090E090930A0180930901A8E2B0E0E8E25B
:10070000F0E0808181608C938FCF809119018823E4
:10071000F1F00E94020380910B0190910C0101966F
:1007200090930C0180930B0180910B0190910C012F
:10073000893C910530F088EC90E090930C01809317
:100740000B018CE291E09093110180931001809154
:10075000100190911101009709F066CF80910B0173
:1007600090910C01009709F45FCF80910B0190915B
:100770000C018430910530F484E090E090930C01FA
:1007800080930B010E948B020E94E20281E0809321
:10079000120180910B0190910C01909304018093C0
:0807A000030142CFF894FFCFE2
:00000001FF
